:100000008CC0B2C0A7C3B0C0AFC0B3C0ADC0ACC09D
:10001000ABC0AAC0A9C0A8C057C1A6C0A5C074459E
:1000200079467D47824887498B60906194629963E5
:100030009D64A265A766AB67B068B469B980BE81EC
:10004000C282C783CB84D084D484FF210000000007
:100050000000000000000000000023456C98C9FF6C
:10006000040714233764A0FFFFFFFFFFFFFFFFFF1C
:10007000FFFFFF00000000000000000023405F7A47
:10008000B4FFFFFFFFFFFF001400081400080E1468
:100090000004080E14000305080E140004080A0EDC
:1000A0001114000305080A0E1014000305080A0EB7
:1000B0001012140008000E00080E0004080E0003C1
:1000C00005080E0004080E1100080E1100F3F404D8
:1000D000080E10121400080A0C0E0F10121400085B
:1000E0000EED14000203040500041400040E1400B5
:1000F000040810140004080F1114000305080A0E68
:100100000004080A0E00EEEDECEB140E08040004E7
:10011000080E00EBECEDEEF3F41411241FBECFE556
:10012000D2E0DEBFCDBF20E0A0E6B0E001C01D926E
:10013000A937B207E1F7EAE7F0E085E5808781E0DB
:10014000838314821282868311828BE0818788E503
:100150008287E0E6F0E08DEF87838EEF8583712C58
:1001600055245A94B2D012C34BCF1BBC19BC18BC37
:100170000895189525B7277E25BF29B7226029BF86
:1001800021E022BF019728F020E188952150E9F76E
:10019000F9CF089588EE93E0EDCF369A3699FECFE9
:1001A00085B10895CF93C72D81E0870D8F73782E89
:1001B000662D90E0DDD26FEF8C2F90E0CF91D8C20A
:1001C000FF920F931F93CF93DF93F82E0BE710E06E
:1001D000CEE7D0E0F11005C0CE01C2D2F801808395
:1001E00004C0F8016081CE01C3D221970F5F1F4F79
:1001F000C437D10579F7DF91CF911F910F91FF900F
:100200000895D0DF81E0DCCF811101C0AECF8150F5
:1002100090E0FC01E45BFF4FE491EBBDFC01E05A90
:10022000FF4FE491E9BDFC01EC58FF4F849188BD7C
:1002300008950F931F93CF93C82F8B01CC2359F0B0
:1002400085E0E2DFC80196DF90DFC80193DFC801D7
:1002500091DFC150F3CFCF911F910F910895EF928D
:10026000FF920F931F93CF93C8E0E82EF12C062F37
:1002700010E084E1C9DFC7017DDF77DFC8017ADFE5
:10028000C150B9F7CF911F910F91FF90EF90089552
:100290001F93CF93DF938FEA87B986EC86B910E17D
:1002A000C0E0D0E085E090E065DF77DFC80FD11DCA
:1002B0001150C1F7CE0124E0969587952A95E1F774
:1002C000DF91CF911F91089518951092790087E7DB
:1002D00090E046D2853519F0612C93DF11C0712C66
:1002E000872D90E03DD2682E8F3F19F080E068DFC7
:1002F00007C0872D91E0970D792E803488F3F6CFD3
:1003000020918300C0917D0010917E0080917B0040
:10031000882319F010E0C0E02AE12F5F90E040E070
:1003200050E0A8E8B0E0222379F0BD016F5F7F4F75
:10033000FB013197E491EE2319F0962F9A1BF6CF2B
:100340002150AD01DB01EFCF092F6C2F70E0A92FF9
:10035000B0E0E02FF0E0112321F09D012E1B3F0BB8
:1003600005C09F0121503109260F371F3197E40F37
:10037000F51FF49027593F4FF901F082015049F7DA
:100380009C0F90938500CC2371F0112329F0292F25
:1003900030E02150310902C020E030E0F901E75996
:1003A000FF4F41E0408327E0290F322F3150E32FE8
:1003B000E91BF0E0ED5EFE4FE491A32FB0E0A759FA
:1003C000BF4FEC933913F2CFE22FF0E0E859FF4F23
:1003D00031E0509169004081541330E0231B209399
:1003E0008600362D353FE8F5452D4D30B0F480912F
:1003F00087008F3F29F4809179008093870006C0A1
:1004000081E0860D682E891708F0612C80918700A5
:100410008F5F8F718093870024C030917900309373
:1004200087004132C0F430918000332311F08823DB
:1004300039F081E0860D682E891798F0612C11C083
:10044000862D6916D9F3662019F08150682E09C0EF
:100450002150622E06C08111F1CF80917C0088234B
:1004600069F3512C8FEF8DBD80E68CBDAB9A8FE385
:1004700084BB8BE187BB88EE88BB81E083BF91EAB8
:100480009ABD80BF8BB780628BBF8AB785608ABFF9
:1004900085B7806285BF789497B986EC86B9C62DFA
:1004A000C53F10F0612C3CC080918700803138F44A
:1004B000E62DF0E0E759FF4FC081DC2F31C06ADE46
:1004C0008091790080938700CBE7D0E000E010E0D6
:1004D000FF24F39481E0800F0F5F1F4F98819F3FAF
:1004E00029F4219608301105A9F7E2CF6DE570E0F7
:1004F000A0DEF801E05AFF4F608088818F25888355
:1005000080DE6FE070E080E294DE88818F25888352
:10051000612C77DE3FDE80917B00882311F3C8CF0A
:1005200041DE10E0F12C81EAE82E96ECD92ECC24A5
:10053000CA94CE3E19F463E481E204C0CD3E21F4B6
:1005400068E284E18CDE6FC0CC3E11F469E203C046
:10055000CB3E19F462E581E0F5CFC33F81F404E0BE
:1005600084E152DE85E090E005DE88E04DDE81E446
:1005700090E000DE0150A1F780ED92E053C0C43F4F
:1005800051F584E690E0F6DD08DE90E0292F30E0BA
:10059000F901E25EFF4FE491E81710F49E5FF6CF99
:1005A000F901E15EFF4F04916DE770E0802F8295C5
:1005B000869587703EDE8EEE92E0DCDD65E070E0D1
:1005C00081E037DE85E694E0D5DD6DE770E0802FD1
:1005D0008F712FDE0DC0CE3F71F400E000938300D9
:1005E00010DE6AEF70E081E024DE0F5F0A31B1F7C0
:1005F000D1DDD0DD18C0CD3F39F58FEF8093840079
:1006000000DE85E001DEC6DDC5DD84E1FDDD40DE26
:1006100080938400F6DDBEDDBDDDF9CFDB30F8F47C
:1006200084EF91E0A7DD8091790080938700B5DDAC
:10063000823808F036C01F5F183008F47ACFD53101
:10064000A8F010E0DAE0CAE08D2FDEDD21DEE7B8A9
:10065000D6B8F39490918400891710F3DFCFF4E1BA
:10066000FF15F0F6C0927900DAE0DACFD23030F040
:100670008D2F86958695D695D80F12C076DD85B7D5
:10068000877E806185BFF89485B7846885BF8B7F3E
:1006900085BF85B7806285BF889585B78F7D85BF0B
:1006A000CD2F10E046CF112416B85FDD87B38C7EC6
:1006B00087BB80E051E041E020E030E0A8E0999B7A
:1006C00006C0F9013197F1F79AB795609ABF96B3D2
:1006D0009A27999B03C0511003C034C0911107C0E1
:1006E00040E2451588F581112FC050E049E0652DA5
:1006F00071E0623208F070E0760F572E511108C099
:10070000811105C081E0911103C080E001C081E04A
:10071000999895B7977E906195BFA895942F9870FA
:1007200011F490E401C090E6916091BD95B7946892
:1007300095BF9B7F95BF78948895F89491B59F7BE2
:1007400091BDBDCF9111D3CF8FE58DBF82E08EBF1C
:100750001FBEBBDD999A552011F0189501C0A3DF8B
:10076000E199FECF9FBB8EBBE09A99278DB3089588
:10077000262FE199FECF1CBA9FBB8EBB2DBB0FB6B7
:10078000F894E29AE19A0FBE01960895F894FFCF8B
:00000001FF
